:020000040000FA
:04000000830105284B
:040004000034003490
:020008000900ED
:06000A00F1014F249321D7
:100010002522C321932193211030F20033224C2258
:100020001F223722502223222B3081212830812188
:100030002E30812137205C20012190239921F20B61
:100040000E2833224C221F221030F2003722502279
:1000500023229921F20B26282B307321283073217B
:100060002E30732137205C200121902321282B3052
:10007000A3222A30C222E3222830C222F0220F30EB
:10008000D822513082223430C222E62255308222D8
:100090003230B5220B30CF22553096220723513013
:1000A0009622E6225B30822208307822E622043053
:1000B000D8222030822208005B3089220F30D10004
:1000C000A030D20051309622E3225D308222652298
:1000D000F0220C30D8225B3082222E30C222F02255
:1000E0000B30D822513082222230B5225D30962248
:1000F000F0220B30D82251309622E622553082224F
:100100002030B5220230CF2255309622E62202302E
:100110007822E6220230D822573082222430B522BB
:100120005D309622F0220D30D822513082222C30C0
:10013000B5225B309622F0221030D8225130962220
:10014000E62202307822E6220230D8228030DD001A
:100150000030DE005D30AC22E6222630C222F022E2
:100160000F30D822593082222830A32257309622CD
:10017000E322C330DD005030DE005D30AC22F022DF
:100180005930AC220723573082220730D82265220B
:10019000F0220B30DD00DE30DE005D30AC22F022DC
:1001A0001030D822513082225730A3220130CF2282
:1001B0006522E330DD004330DE005D308922F0222D
:1001C0001030D82251309622E6220E30DD00CF309A
:1001D000DE005D309622E6220430D82265225730B8
:1001E000A3220130CF22E6220A30782207230730EB
:1001F000DD00D030DE005D30AC22E32222308222EE
:1002000008002E30A32214307822F0224B307822BE
:10021000F022652201306E220A30CF22E6220B3016
:10022000D822513082222E30A32214307822F0229C
:100230000530D8226522F0222B307822F022652268
:1002400001306E221230CF22E6221330D8225330F2
:1002500082225130892229307822E322533096229B
:10026000E3220130D822243082222030892200303B
:10027000DD00FA30DE005D309622E322513082222A
:1002800032307822B61BE322B61FE6226430782291
:10029000072353308222513089222E309622F022B9
:1002A0003030DD00D430DE005D309622072353303D
:1002B0009622E62224309622E62224308222A41BB3
:1002C000702965220330DD00E730DE005D308922D1
:1002D000E322B31F08000330A400E730A5000800A4
:1002E000A401A501080084000430D000840A840A17
:1002F0000310800D8403800D8403800DD00B7629BC
:1003000008008400840A000884038000840A840AA8
:100310000008840380000800633081000B11640032
:100320000B1D902908006430D0008C21D00B95293A
:100330000800163098006400630063000800103065
:100340009800640063001630980064000800D00034
:1003500083169C18A9298312700883169B008312A8
:10036000500883169A001C1555309D00AA309D0038
:100370009C141C1183120800700883169B001C1427
:100380001A0883120800C621CA21080005100800B7
:10039000051408008316851483120800851083163F
:1003A000851083120800CA21C821CE21C621C82188
:1003B000CA21C6210800C821C6210800CA2103108D
:1003C00085180314DB29CE21DB21CA29CA21DB29A8
:1003D000851CE8299F218518EA290800031CCE21E5
:1003E0000318CA21DB29851C031085180314DB2997
:1003F000A7000830A600A70DEE21A60BFB290800D8
:10040000A7010830A600F321A70DA60B032A270891
:100410000800D321F821DE2103181E2AE82100223A
:10042000F300E3210022F400E6217408B00773080A
:100430000318730FAF070318AE0A08000800AE01D7
:10044000AF01B00108000530092A262AAA30C600EB
:100450002030F0001630B1007024A721C60AF00A3F
:10046000B10B2C2A0800AB01AC01AD010800F4303F
:10047000C6002E3061249F21F630C6000230C7002E
:100480007330840080247408AD0773080318730F59
:10049000AC070318AB0A0034A801A901AA0108009F
:1004A000F430C600343061249F21F630C60002309B
:1004B000C7007330840080247408AA0773080318E7
:1004C000730FA9070318A80A00343308B7003408CB
:1004D000B8003508B9003608BA000800B301B40105
:1004E000B501B600B61F0800B303B403B503080096
:1004F000B701B801B901BA00BA1F0800B703B803C1
:10050000B9030800840035088000840A360880009A
:100510000800B301B40184000008B500840A000893
:10052000B600B51F0800B303B4030800B701B80153
:1005300084000008B900840A0008BA00B91F080046
:10054000B703B8030800B301B40184000008B50084
:10055000840A0008B6000800B701B801840000084A
:10056000B900840A0008BA000800B301B401F00021
:10057000BC21B500F00ABC21B600B51F0800B303CA
:10058000B4030800B701B801F000BC21B900F00ABB
:10059000BC21BA00B91F0800B703B8030800C000A7
:1005A0000310B60DB50DB40DB30DC00BD02A080065
:1005B000C0000310B30CB40CB50CB60C331BB3174E
:1005C000C00BD92A08007723031808003308370620
:1005D000BF004023031037083306BF1F803E0800CA
:1005E000BF016123031C7423031808004F235C23FD
:1005F0001F30C00087233E0D03184023031C330D1A
:1006000003180800C00BFA2A3F1864230800BF0132
:100610003A08390438043704003C031C6123031CE6
:10062000742303180800BB01BC01BD01BE01872370
:100630001F30C000872337083E02031D292B3808CE
:100640003D02031D292B39083C02031D292B3A08C2
:100650003B02031C3B2B3A08BB023908031C390F31
:10066000BC023808031C380FBD023708031C370FC3
:10067000BE0203103614C00B1A2B3F186423080067
:100680003A08B60739080318390FB50738080318B0
:10069000380FB40737080318370FB30708003608B8
:1006A000BB003508BC003408BD003308BE0008009C
:1006B000BA01B901B801B701B601B501B401B3017E
:1006C0000800330D031C080033088039B609B5094A
:1006D000B409B309B60F712BB50F712BB40F712B81
:1006E000B30ABF0A33070800370D031C0800370898
:1006F0008039BA09B909B809B709BA0F842BB90FFB
:10070000842BB80F842BB70ABF0A37070800B60D31
:10071000B50DB40DB30DBB0DBC0DBD0DBE0D080068
:100720000430DF000330E000A01F9D2BA109A009C9
:100730000130A1070318A007E01520302C2475080C
:100740000F39D500760E0F39D60076080F39D7004D
:1007500024302C2475080F39D800760E0F39D900B3
:1007600076080F39DA0022302C24750E0F39DB00A1
:1007700075080F39DC00760E0F39DD0076080F3969
:10078000DE00C22B03015F066006570656065506BB
:100790005A06590658065D065C065B065E06E100D1
:1007A00005305F0760075707560755075A0759076F
:1007B00058075D075C075B075E0761070F39E200BA
:1007C00003011224030112241B241B2420245F088C
:1007D00012242024600812242024570812242024E4
:1007E0005608122420245508122420245A081224C2
:1007F00020245908122420245808122420245D089B
:10080000122420245C08122420245B0812242024B3
:100810005E08122420246108122420246208122475
:1008200020240800D300172417241724172CD30CD6
:100830000318202C1B2C0515252425240511252CF7
:100840000515252405112524252C6230D400282CDB
:100850000000D40B282C0800D000D00A0310103060
:10086000D200F501F60150088400800D8403800D4C
:10087000F60DF50DD20B3D2C080076308400442493
:10088000753084004424332C03300007D100D11983
:10089000800030300007D100D11B800008008501A6
:1008A0000730990083168530810099019F016130DE
:1008B0008F00383085008B018312163098000511A7
:1008C0000800C500D424DF244318982CE8244318DA
:1008D000982C4508AB24BC244318982CDA24080033
:1008E000D424DF244318982CE8244318982CD424CB
:1008F000E3244318982C9A24C724DA2444080800D7
:10090000D424DF244318982CE8244318982CD424AA
:10091000E3244318982C9A2444088000840AC70BC7
:10092000922C942CD1248B2CC724DA244408080060
:10093000DA240800C4010830C200EF24F824851E20
:10094000A22CA52C0310C40DA72C0314C40DFC2449
:10095000C20B9E2C0800C1000830C2000310C10D5C
:10096000031CB32CB72CF324EC24EF24B92CEF2474
:10097000EC24C20BAE2C0800EF24F824C201C20AFA
:100980000319CF2C851ABF2C4310FC240800EF2438
:10099000EC240800D424DF244318CA2C0800431494
:1009A0000800F324EC240800FC24EF24F824F324AA
:1009B000FC240800FC24F324F824EF240800EE3083
:1009C000AB24BC240800EE300138AB24BC24080062
:1009D0004608AB24BC240800F824FC240800831635
:1009E000851683120800851283168512831208006B
:1009F000831605168312080005128316051283124A
:020A00000800EC
:02400E00CC30B4
:00000001FF
